:100000000C9434000C943E000C943E000C943E0082
:100010000C943E000C943E000C943E000C943E0068
:100020000C943E000C943E000C943E000C943E0058
:100030000C943E000C943E000C943E000C943E0048
:100040000C943E000C943E000C943E000C943E0038
:100050000C943E000C943E000C943E000C943E0028
:100060000C943E000C943E0011241FBECFEFD8E04C
:10007000DEBFCDBF0E9440000C9477020C940000BC
:1000800081E087B988B9000000000000000000008E
:10009000000018B800000000000000000000000090
:1000A0000000000000000000000000000000000050
:1000B000000088B9000000000000000000000000FF
:1000C00018B8000000000000000000000000000060
:1000D0000000000000000000000000000000000020
:1000E00088B900000000000000000000000018B8FF
:1000F0000000000000000000000000000000000000
:10010000000000000000000000000000000088B9AE
:1001100000000000000000000000000018B800000F
:1001200000000000000000000000000000000000CF
:1001300000000000000000000000000088B900007E
:100140000000000000000000000018B800000000DF
:10015000000000000000000000000000000000009F
:100160000000000000000000000088B9000000004E
:10017000000000000000000018B8000000000000AF
:10018000000000000000000000000000000000006F
:10019000000000000000000088B90000000000001E
:1001A00000000000000018B800000000000000007F
:1001B000000000000000000000000000000000003F
:1001C00000000000000088B90000000000000000EE
:1001D0000000000018B8000000000000000000004F
:1001E000000000000000000000000000000000000F
:1001F0000000000088B900000000000000000000BE
:10020000000018B80000000000000000000000001E
:1002100000000000000000000000000000000000DE
:10022000000088B90000000000000000000000008D
:1002300018B80000000000000000000000000000EE
:1002400000000000000000000000000000000000AE
:1002500088B900000000000000000000000018B88D
:10026000000000000000000000000000000000008E
:10027000000000000000000000000000000088B93D
:1002800000000000000000000000000018B800009E
:10029000000000000000000000000000000000005E
:1002A00000000000000000000000000088B900000D
:1002B0000000000000000000000018B8000000006E
:1002C000000000000000000000000000000000002E
:1002D0000000000000000000000088B900000000DD
:1002E000000000000000000018B80000000000003E
:1002F00000000000000000000000000000000000FE
:10030000000000000000000088B9000000000000AC
:1003100000000000000018B800000000000000000D
:1003200000000000000000000000000000000000CD
:1003300000000000000088B900000000000000007C
:100340000000000018B800000000000000000000DD
:10035000000000000000000000000000000000009D
:100360000000000088B9000000000000000000004C
:10037000000000000000000000000000000000007D
:10038000000018B80000000000000000000000009D
:100390000000000088B9000000000000000000001C
:1003A000000000000000000000000000000000004D
:1003B000000018B80000000000000000000000006D
:1003C0000000000088B900000000000000000000EC
:1003D000000000000000000000000000000000001D
:1003E000000018B80000000000000000000000003D
:1003F0000000000088B900000000000000000000BC
:1004000000000000000000000000000000000000EC
:10041000000018B80000000000000000000000000C
:100420000000000088B9000000000000000000008B
:1004300000000000000000000000000000000000BC
:10044000000018B8000000000000000000000000DC
:100450000000000088B9000000000000000000005B
:10046000000000000000000000000000000000008C
:10047000000018B8000000000000000000000000AC
:100480000000000088B9000000000000000000002B
:10049000000000000000000000000000000000005C
:1004A000000018B80000000000000000000000007C
:1004B0000000000088B900000000000000000000FB
:1004C000000000000000000000000000000000002C
:1004D000000018B80000000000000000000000004C
:1004E0000000000090E19A95F1F700C0CBCDF894A0
:0204F000FFCF3C
:00000001FF
